:020000020000FC
:0200000006C038
:10000C0034C00FE70ABB0FEF0BBB0FEF07BB0FEFB3
:10001C0008BB0FE004BB0FE305BB0FEF01BB0FEFF9
:10002C0002BB0FE50DBF04E00EBF8FEF9EE120E099
:10003C0030E040E050E060E070E000E808B9F8948F
:10004C0000E009BF08E002BD0AE005BD0FE103BDF9
:10005C0002B507700030E1F700EC08BF00E809BFFB
:10006C0000E705BF78948895FECF41D080FF1BD068
:10007C008A9521F49A9511F49EE101D01895239557
:10008C002A3081F420E03395363061F430E043952A
:10009C004A3011F440E05395443021F4523011F4BD
:1000AC0040E050E00895703009F07A9503B3007386
:1000BC00601751F0703041F405FF03C004FF03C01A
:1000CC0003C008D001C008D0602F05FF74E004FF06
:1000DC0074E00895DCDF089523952A3029F420E09C
:1000EC003395363009F430E08FEF9EE10895052FFB
:1000FC0043D080FD0095006305BB042F13D000682E
:10010C0080FD009502BB032F0DD080FD00950BBB2D
:10011C00022F08D086FD0F7786FF006880FD0095C2
:10012C0008BB08950030A1F00130A1F00230A1F01D
:10013C000330A1F00430A1F00530A1F00630A1F09D
:10014C000730A1F00830A1F00930A1F00FEB0895B1
:10015C0000EC089509EF089504EA089500EB089562
:10016C0009E9089502E9089502E8089508EF089551
:10017C0000E8089500E90895013021F0023021F0E3
:0C018C000FEF089509EF08950CEF08959F
:00000001FF
